:020000040800F2
:10000000C03B002009170008053D0008F516000850
:10001000F5160008F5160008F516000800000000A7
:100020000000000000000000000000006117000850
:10003000F516000800000000011900084921000819
:100040007919000879190008791900087919000848
:100050007919000879190008791900087919000838
:100060007919000879190008791900087919000828
:100070007919000879190008791900087919000818
:100080007919000879190008791900087919000808
:1000900079190008791900087919000879190008F8
:1000A00079190008791900087919000879190008E8
:1000B00079190008791900087919000879190008D8
:1000C00079190008791900087919000879190008C8
:1000D00079190008791900087919000879190008B8
:1000E00079190008791900087919000879190008A8
:1000F0007919000879190008791900087919000898
:100100007919000879190008791900087919000887
:100110007919000879190008791900087919000877
:100120007919000879190008791900087919000867
:100130007919000879190008791900087919000857
:100140007919000879190008791900087919000847
:100150007919000879190008791900087919000837
:100160007919000879190008791900087919000827
:100170007919000879190008791900087919000817
:100180007919000879190008791900087919000807
:1001900079190008791900087919000879190008F7
:1001A00079190008791900087919000879190008E7
:1001B00030B587B003F052F903F051F925484921D1
:1001C00003F05EF903F049F903A800F0A7FC224B05
:1001D0001B68834204D02148452103F051F9FEE712
:1001E000059A1F48492103F04BF903991D484B7D9F
:1001F0000A7DC98A0091492103F042F91A48492130
:1002000003F03EF99DF8100002A900F033F804460F
:1002100000B1FEE7029A059B144D1344039A12891C
:1002200013442B6004F04AF801F09CF801F086FAC0
:100230002B681B6883F3088884F31488BFF36F8FDF
:10024000BFF36F8F2B685B6898470948452103F01F
:1002500017F9FEE7C64C000894030020DF4C0008A5
:10026000024D0008314D00084F4D000808020020E3
:10027000744D000808B5024618B94FF000630B60D2
:1002800008BD0348452103F0FBF86FF01500F7E7C0
:10029000974D000821B1012906D06FF01500704775
:1002A000044B53F830007047024B03EBC00358680F
:1002B000704700BFDC4A000808B5024803F0D2F8D6
:1002C000002008BDB04D0008014B1B68184700BF57
:1002D0000000002030B5044685B00D4610220021F4
:1002E000684604F0F1F902238DF802302A46044BE7
:1002F00001932146684602F057FF05B030BD00BFAC
:10030000C9020008034A536823F002035360002027
:10031000704700BF002004E0EFF31180102383F347
:100320001288BFF36F8F094B1A683AB9084A1168EF
:1003300041F4807111601168C905FCD51A68013259
:100340001A6080F31188BFF36F8F7047100200208E
:1003500000700040EFF31180102383F31288BFF385
:100360006F8F114B1A689AB9BFF35B8F0F4B012245
:1003700053E8001F002904D143E8002CBCF1000F12
:10038000F6D1BFF35B8F80F31188BFF36F8F704797
:10039000012A01BF06490A6822F480720A601A68BD
:1003A000013A1A60EFE700BF100200200C020020A3
:1003B00000700040134B1A6842F4007282B01A6059
:1003C0001A6842F480621A601A6842F480721A60F5
:1003D0000D4B0E4A1A600E4A536843F001035360F6
:1003E0000C4B9A6D42F080529A659B6D0A4A03F05D
:1003F00080530193019B936843F48043936002B060
:10040000704700BF002002402C0000200024F400B0
:10041000002004E00010024000700040014B036027
:1004200000207047E44A000870B5104B1C680D4668
:10043000B4B10F4B196800238B4202DB6FF001004F
:1004400070BD224612F8106B864202D0013314466A
:10045000F2E7E06804F009F828B12C600020EFE72B
:100460006FF00C00ECE76FF01200E9E704000020E9
:10047000E44A000810B588B0436802938368C068F6
:10048000CDE903320A680023CDE906230C4601AA10
:100490000449059303F070FD079808B9059B236094
:1004A00008B010BD5535000880B505460E46174604
:1004B000984602F083FC034601F070FADFF81890CA
:1004C000044649F80030424630463946A84754F8B9
:1004D000090001F0FFF900BF080000002DE9F04F0E
:1004E0009DB0DFF8E480289FD8F800400397279F4D
:1004F00002970DF1500B269FCDF804B00097299D6F
:1005000081468A46164603F060F828B1D8F80040C4
:1005100020461DB0BDE8F08F55B15A46134603CBB7
:1005200069601CA98B4228601A4605F10805F5D1BF
:100530000023009332464FF6FF73514606A803F09E
:100540007BF805460028E1D1314648460B9F03F071
:1005500046F9B842DAD30DF1120304AA05A906A898
:1005600003F0B8F80028D1DB2AD1059906A803F0DA
:10057000FCF8BDF8123040B914494FF6FF7031F85D
:10058000022B8242C2D09A42F9D1102BE3D1BDF89E
:100590001040202CBAD1059923460CAA304602F00F
:1005A0008AFF0028B2D122460CA9584603F0EBF886
:1005B0000446074B1B6898424FF00105CBD0A5E7D6
:1005C000012DA3D1A4E700BF0C000020984C000827
:1005D00094030020084A0B78400052F820108B4208
:1005E00008D0013052F8200083420CBF48204FF061
:1005F000FF30704748207047284B00081FB558232C
:1006000003FB01006A46046AA168102310392046E2
:1006100002F051FF034628B122780448452102F038
:100620002FFF0024204604B010BD00BFE94D000894
:1006300038B50E4B002918BF0B464362C033036523
:100640000121044603F012F958B90221204603F0B3
:100650000DF9054638B9206A02F06CFFE0652846BE
:1006600038BD0125FBE70925F9E700BF140200208A
:1006700010B52C2359434218146A0CB903F074FBCB
:1006800041580D4B994206D1D16813895B1802D2AB
:100690005189C91801D300200CE0A3689942FAD20D
:1006A000106920F4F97020F001000005000DB0FA87
:1006B00080F0400910BD00BF3DB8F3961FB52C2354
:1006C00003FB02010A6A0AB903F04EFB0023CDE9DD
:1006D000023301934FF480730093034BFFF7FEFE48
:1006E00005B05DF804FB00BFD80800202DE9F041FB
:1006F0002C2707FB01070546D7F820800C46164635
:10070000B8F1000F01D103F02FFB03F039F910B954
:100710003B69DB061DD5C4B14146284603F0B5F957
:10072000F379042B0CD1296A0029ECD0284603F078
:10073000ACF9024648B91748492102F0A1FE04E08D
:10074000002001F0E7FE0428EDD0134B1868BDE847
:10075000F08121462846FFF78BFFA8B90F4B186898
:100760000F4B1B688342F2D00E4A0F4B0F48002CF0
:1007700018BF1A46452102F083FE002CE5D0012166
:10078000404603F0F8F8E0E7224631462846FFF7F6
:1007900095FFE5E7274E0008080000200C00002028
:1007A00094030020154E00081D4E0008664E0008F8
:1007B00073B50D46044600212846CDE9001103F02B
:1007C0002FF950B323681E4EB34206D101AA20462A
:1007D00003F007F808B103F0C7FAE36AB34206D1A1
:1007E0006A460121204602F0FCFF0028F3D1DDE932
:1007F00000239A4284BF13460192AB60019A2946B6
:10080000204600F091FB0F4B1A68002A03DD0E48CA
:10081000572102F035FE02B070BD01462046FFF7B9
:10082000EDFE06460028D6D005F1080102F0BAFF19
:100830000028D0D1AB680193304602F03BFEDDE7E3
:100840003DB8F396F80700208E4E00082DE9F843D6
:10085000099F0E46904699460024BC4201D30020D1
:100860000EE03D1BB5F5806F28BF4FF480650C4A44
:100870002B4604EB0901304602F01DFE10B10120A9
:10088000BDE8F8830899064A2B466118404602F0F5
:1008900027FE0028F3D12C4402F0E1FDDDE700BF84
:1008A000980300202DE9F04186B00E46044603F07F
:1008B0008EF8014620B19048452102F0E1FDFEE7A7
:1008C0002046FFF7B5FE054678B9002211462046BE
:1008D00003F063F8054610B388480022572102F060
:1008E000CFFD012384F8583009E0854818225721AC
:1008F00002F0C6FD01239D4284F85830E5D194F8FA
:1009000058308DF80F30042B00F29180012B00F24B
:10091000968000F0AC80FF2384F85830A7E0204692
:1009200000F000FA0028DCD0764B012702A920460F
:10093000CDE90273CDE9045503F0E5F838B172480A
:100940002A46572102F09CFD84F85870D7E702A888
:1009500003F066F880F0010102AAC9B2204603F054
:100960001CF805460028B7D102A803F059F898BB37
:1009700002A92046FFF71CFF9DF80F3084F858307D
:10098000033B012B07D8284600F0F0F8054610B1CC
:10099000FF2384F858309DF80F30023B022B0DD80E
:1009A000002000F0CDF8054640B1FF2384F8583010
:1009B0005648452102F064FD03F0D6F994F858300A
:1009C000FF2BF5D0002DF7D12A462946204602F00C
:1009D000E4FF002885D0EFE79DF80F80B8F1010F04
:1009E00018D1284601F096FD831E022B05460ED82D
:1009F00002AA41462046FFF779FE454B1B68984204
:100A000005D0444B1D68A84214BF0525012584F874
:100A1000585074E702AA39462046FFF767FE3C4B60
:100A20001B6898420CBF9DF80F3005235AE7052B31
:100A30007FF471AF002000F099F8C0B16BE702A914
:100A40002046FFF7B5FE94F85830DA1E012A0BD87D
:100A5000002000F08BF818B9002000F071F830B1D8
:100A6000FF2384F85830A7E7023B012BF4D994F810
:100A70005830FF2B9CD00022012B274F019211D020
:100A80001146204602F089FF60B13D681022002126
:100A900002A803F019FE204602F0B1FF284606B076
:100AA000BDE8F081002211462046FFF71FFEDFF867
:100AB00060803D68D8F800309842E7D1A842E5D080
:100AC000144B1B689842E1D00021204602F07DFFC4
:100AD0000028DAD1019B01330193019B012B00D047
:100AE000FEE7206A02F099FC3071236A5B6834608B
:100AF000D8F80050B360C9E7BD4E0008304F000879
:100B0000EE4E0008010100015C4F0008864F00080E
:100B100094030020080000200C00002010B50446BB
:100B2000064802F079FF05482146FFF7BBFE044660
:100B3000024802F0B5FE204610BD00BF9807002015
:100B400013B5094B01A913F83000FFF76DFC48B944
:100B5000019803F06AFC0446019802F0ABFC2046C1
:100B600002B010BD0124FAE7304B00081FB50F4B4F
:100B700001A913F83000FFF757FCA8B9019802A9A2
:100B800001F072FC044668B99DF80B30032B03D1C9
:100B9000019803F012FC0446019802F08BFC2046F9
:100BA00004B010BD0124F7E70124F8E7304B00083A
:100BB0002DE9F34106460C4617461D460BB90021A8
:100BC00021E0184602F02CFF01460028F7D13046FC
:100BD000FFF714FD18B9012002B0BDE8F08101A9AA
:100BE00002F0E0FD0028F6D10199304602F0BDFF89
:100BF000736A59686B79012B0CD1002CDFD12B68FB
:100C0000834298BF00212C2303FB0466306AB0B9ED
:100C100003F0AAF8022BD2D12B68012B05D983420D
:100C2000CDD8B4FA84F46409C9E7C8D1002CEAD05D
:100C3000012CC4D12C79023C18BF0124BFE720232A
:100C40003A4602F038FC0028C5D1002DC4D03868DF
:100C5000024BC01A18BF4FF0FF30BDE73DB8F39606
:100C60002DE9F04F074685B00C4601460020164698
:100C7000FFF7B0FC051E4FDB3846D4F85C9002F05D
:100C800084FD4FF0000800904FF0010A4FF0FF3450
:100C90005FFA89F99DB9B8F1010F03DD20484521BC
:100CA00002F0EEFB631C06D0172C2ADC013440F264
:100CB00001133460B380284605B0BDE8F08F009979
:100CC00005F1FF3B01230DF10F020BFB0911384623
:100CD00002F0F1FB031E019320DB01220DF10F0155
:100CE000384603F006FB019B30B1534501D008F1B3
:100CF00001085D469A46CDE7B4F1FF3F08BF2C4698
:100D0000F7E70223183C7371631004F00104013308
:100D1000013433603471CEE70725CCE70125CAE7FB
:100D2000924F0008F8B5866A456DAE42044608D079
:100D30006B1CB34205D01748572102F0A1FB0020DD
:100D4000F8BD182E19D914485721F6E7626A02EB4C
:100D5000C3025768226D02EBC3025268974202D069
:100D60000E485721E9E701339D42EFD1204602F0BA
:100D7000ADFF28B90A485721DFE700231F46F3E7F4
:100D8000AE4205D9636A03EBC5035B68BB42E7D19A
:100D90000120D5E7B54F0008ED4F00081C500008B2
:100DA0004850000810B588B0044604A9006A01F054
:100DB0005BFB08B102F0D8FF9DF81020012A44D057
:100DC000264B2749032A08BF0B469DF813200292A1
:100DD0009DF8122001929DF811202248009249218D
:100DE000214A02F04DFBE06C06A901F03DFB0446F0
:100DF0000028DFD19DF81820012A28D0174B184968
:100E0000032A08BF0B469DF81B2002929DF81A206A
:100E100001929DF8192000921248144A492102F0CB
:100E20002FFB9DF81030012B13D19DF81230032BAE
:100E30000FD19DF81830012B0BD00D48492102F03D
:100E40001FFB0224204608B010BD0A4BBDE7094B2A
:100E5000D9E70948492102F013FBF3E78150000864
:100E60008A5000089E50000890500008DF5000088B
:100E7000EF500008855000080E51000870B54B680F
:100E80001446234A03F0FF23934286B006460D46DC
:100E90003AD10B68012B37D104A9204601F0E4FABE
:100EA00008B102F061FF9DF81020012A2ED0194BE5
:100EB0001949032A08BF0B469DF8132002929DF89A
:100EC000122001929DF8112000921448144A4921E1
:100ED00002F0D6FA9DF81030032B15D1214630468A
:100EE00002F0D3FD0028DCD1204603F066FA00288A
:100EF000D7D1A968204602F063FC0028D1D1204652
:100F000001F090FA0028CCD106B070BD054BD3E7B4
:100F100000010004815000088A5000089E5000081B
:100F2000DF500008855000082DE9F04F164687B0C5
:100F300005460C467C48492102F0A2FA3146284673
:100F400002F013FE6B6A804620465E6802F068FD80
:100F5000E8B1E86D02F0A5FCAF6A0023013F33441D
:100F6000984201D9013FFAE7B84510D36F4857219D
:100F700002F086FA07FB06F36D4808FB066257216C
:100F800002F07EFA0123E37107B0BDE8F08F2F6A0B
:100F90000FB902F0E9FEEB6C0393002BF9D01A466F
:100FA00021462846FFF76AFF6379012B54D1DFF809
:100FB00084B1C1464BE02268C2F101034344994524
:100FC00043D86B6A196853F8390003EBC903012A47
:100FD00053F8083CA3EB0103A0EB010A049315D1DD
:100FE000E368022B0CD03946284602F04EFD00285B
:100FF000CFD122463946284602F05CFD0028C8D1F0
:101000000399284602F041FD0028C2D10023324650
:101010005146384602F064FC0028BAD1CDE900A65A
:10102000049B3A4639462846FFF710FC0028B0D109
:101030002146284602F001FD23680133236020B1D8
:10104000DBF800300133CBF8003009F1FF39B9F19A
:10105000000FB0D101232360022363714FF0010917
:10106000C84591D3236899455AD36A6A4FEAC903A0
:1010700052F839100491083B296DD2F800B0C858D5
:101080000968A0EB010A2179012947D1D1583846D6
:10109000A1EB0B0100233246059102F021FC002850
:1010A0007FF477AF059900910196039953463A462C
:1010B0002846FFF7CBFB00287FF46BAF214628467C
:1010C00002F0BBFC0223237118B11A4A13680133E2
:1010D0001360039800233246514602F001FC0028B9
:1010E0007FF457AF049B039ACDE900A6A3EB0B0353
:1010F00039462846FFF7AAFB00287FF44AAF21466D
:10110000284602F09AFC23680133236001232371EF
:1011100030B1084A13680133136001E00229D8D0C6
:1011200009F101099CE700BF255100084E51000854
:101130007D510008F80700202DE9F04F9DB00368AD
:1011400002934368039383680493C3680593036918
:1011500006934369079383690893C36909938A4691
:10116000DDE9062CDDE904B7DDE902159846DFF874
:1011700094E1089B009300265AF806405EF8049B11
:101180000CAB24BA9C514FEAF223A14483EAB21378
:10119000009C83EA72634B4424EA020402EA0C09CD
:1011A00084EA09042344434485EA0B044FEA713876
:1011B00088EAB1080C4005EA0B0984EA090488EAC8
:1011C000B1580436A044402E03EB070443445F4665
:1011D000DDF8008040F087804B4E0A964FF0100AF1
:1011E00056460AF1010A0DF1700E0AF00F070EEBD8
:1011F000870706F00F0957F8407C01974FEAB74878
:1012000088EAF71806F10E0707F00F070EEB8707BD
:10121000093657F8407C4FEAF74E8EEA774ECDF804
:101220002CE006F00F060DF1700E0EEB86060EEBAD
:10123000890956F8406C59F840EC7644DDF804E032
:1012400088EADE08DDF82CE046448EEA972E7644E4
:1012500004EA02084FEAF42E2CEA040787EA08079A
:101260008EEAB41EDDF8288049F8406C8EEA746E70
:10127000774458F804EFCDF8288077443744009E2F
:10128000CDF800C03E444FEA733E81EA05078EEA7E
:10129000B30E1F4001EA05088EEAB35E87EA08072D
:1012A0007744BAF1400F06EB0B0E3744AB4622D120
:1012B000029E3E440660039E1E44049B46600B440F
:1012C0008360059B2B44C360069B73440361079BAB
:1012D00023444361089B13448361099B6344C361B6
:1012E0001DB0BDE8F08FCDF800C0AB4694460D466A
:1012F0002246194640E794460D4622461946744652
:101300003B466DE7384B0008744B000810B50446A7
:10131000C8B17022002102F0D7FC0B4B0B4A0C49DC
:101320000C48C4E900230C4BC4E902130B4BC4E97D
:1013300004030B4BA36103F17453A3F52303A3F63A
:101340009243E361012010BD85AE67BB67E6096A81
:1013500072F36E3C7F520E513AF54FA58C68059B97
:10136000ABD9831FBFF36F8F72B6124B4FF0FF32B2
:10137000C3F88020C3F88420C3F88820C3F88C20E9
:10138000C3F89020C3F89420C3F89820C3F89C2099
:10139000C3F88021C3F88421C3F88821C3F88C21C5
:1013A000C3F89021C3F89421C3F89821C3F89C2175
:1013B000704700BF00E100E008B50348034A002180
:1013C000121A02F091FC08BD58000020DC09002030
:1013D0000748084A084908B5121A02F087FC07486E
:1013E000074A0849BDE80840121A02F07FBC00BF56
:1013F00000000020540000200053000800000020DE
:10140000000000200053000830BFFFF7FDBF00BF01
:101410002DE9F0410B4EDFF8308006EB0807CC1BBE
:10142000054632460949204603F040F9A0194246D4
:101430000021083C03F048F92C6707F10800BDE8DB
:10144000F08100BF0000000004000000D44A000842
:1014500070B5264B15469A6A12F0100F9A6A14BF9F
:101460001124102412F0080F9A6A18BF1224920750
:1014700006460AD5586B9A6A140634D519B19A6A89
:1014800022F080029A62132401E06FF01500174BDE
:101490009A6A12F0010F9A6A18BF142412F0200FF2
:1014A0009A6A18BF1524D20602D49B6A9B070AD5F4
:1014B0000E4B5B68190506D5314600F0C1F910B135
:1014C00080F309880224094B9A6A920642BF5A6A3D
:1014D00022F400525A629A6A42F0FF029A62002392
:1014E0002B70204670BD6FF01500CCE700ED00E0DA
:1014F000134B9A6A12F0007F9A6A14BF1E201D20B7
:1015000012F0807F9A6A18BF1F2012F4002F9A6A87
:1015100018BF212012F4802F9A6A18BF222012F4DB
:10152000003F9A6A18BF232012F4803F9A6A6FEA3C
:1015300002426FEA12429A6218BF2420704700BF2D
:1015400000ED00E010B5194B0246986A9C6A10F451
:10155000805F14BF1720162014F4006F9C6A18BF18
:101560001820A40509D5986B986A000404D51AB10F
:101570009A6A22F400429A6219200C4B9A6A12F479
:10158000806F9A6A18BF1A20D2050CD49B6A13F494
:10159000005F18BF1C20054A936A43F47F4393629F
:1015A00000230B7010BD1B20F5E700BF00ED00E02D
:1015B000F0B5494B5B688BB00446C3F308030025C4
:1015C00085F31188BFF36F8F02F07F40B0F17F4F3A
:1015D00011D102F00C0008280DD010074CBF0C46AA
:1015E00001250022033B8DF80720032B05D8DFE8F7
:1015F00003F024686C652C46F3E700239DF8072070
:10160000CAB902AE04F1200720686168324603C2FD
:101610000834BC421646F7D1099A002D59D0C2F3BE
:10162000080121B96FEA52226FEA4222099202A907
:10163000184602F05DFB0BB0F0BD274BDA6A91074C
:10164000DBD4DA6A002AD8DBDA6A5200D5D55A69C7
:10165000A16942F480725A61BFF34F8FBFF36F8F5D
:1016600031F8022C596921F480715961BFF34F8F11
:10167000BFF36F8F02F47F43B3F55F4F04D1D2B253
:10168000022A01D12368B9E7134B9A6AD2B23AB160
:101690000DF1070201212046FFF7DAFE0346ADE710
:1016A0009A6A12F47F4F05D00DF107010120FFF770
:1016B00049FFF3E79B6AB3F5803F9ED3FFF718FF1E
:1016C000ECE70DF107020021E5E70DF1070100202D
:1016D000EDE76FF30802A9E700ED00E0044B5A695B
:1016E00042F010025A615A6922F008025A617047AA
:1016F00000ED00E0EFF30880EFF3098101B57246D9
:10170000FFF756FF01BD00BF0A4880F3088810208C
:1017100080F3118808484FF40461401880F3098869
:10172000EFF314800221084380F31488BFF36F8F16
:1017300000F04EF8C03B0020000A00200749D1F815
:1017400090200023C2F307221846934200DB704723
:10175000C1F89830C1F8A0000133F6E700ED00E0D1
:101760001EF0040F0CBFEFF30880EFF309808169CE
:1017700011F8021C0229FFD001B5724602F0BEFA30
:1017800001BD00BF40B20028A8BF00F1604001F1D8
:101790000101B8BF064B4FEA0111ACBF00F5614033
:1017A00000F00F00C9B2B4BF195480F8001370479D
:1017B00014ED00E0044B054A23F07F039360BFF370
:1017C0004F8FBFF36F8F70470000000800ED00E0FF
:1017D00008B5FFF7EFFF0B4AD2F8883023F4700307
:1017E000C2F88830EFF3148323F0040383F31488E2
:1017F000BFF36F8FFFF7E0FDFFF7EAFD00F0B0F8F1
:1018000000F0C4FF00ED00E042F8203C009B42F8ED
:101810001C3C0A49019B42F8183C029B42F8143CCC
:1018200021F001014FF0807342F8043C42F8081C9B
:101830000023203A02654367704700BFA9040008EF
:10184000094A0346906870B113F1160F006E05D077
:10185000A0F14002934205D3834203D2814228BFC4
:101860000020704700207047AC08002008B51546DE
:101870000B4A0C4B9060026F1A600E4600F0A0F805
:101880002C4686F309880020034B98472046002108
:1018900000220023014C2047213D0008A904000834
:1018A000AC080020FC070020014B10221A61704791
:1018B00000ED00E0054B5A699B689A421FBF044A3D
:1018C000536843F080535360704700BFAC0800205A
:1018D00000ED00E0084B9B6883420BD1EFF30583DA
:1018E00043B1064B5A6842F080525A605A6A22F459
:1018F00000425A6202F0E6BDAC08002000ED00E0B4
:1019000014498A684FF030001044EFF3098C80E8E6
:10191000F01F102080F31288BFF36F8F0E4F4FF02F
:1019200000664A698A603E60106F0C4C2060506F00
:101930000023536780F3118804B5104600F040F887
:10194000BDE8044002F1300090E8F01F8CF30988F4
:1019500070470000AC08002004ED00E0FC07002008
:10196000044800231021C21801335C2B82F80013B5
:10197000F9D1704700E100E008B5EFF30583064AAE
:10198000103B02EBC30152F8330049688847BDE8B9
:101990000840FFF78FBF00BFB84700080148006844
:1019A00070470000FC070020024B034A0348012156
:1019B00000F076B80080002000000020384C0008BD
:1019C000036E054A403B1360044B4021C2E90113FA
:1019D0001046012100F06EB80008002000000B1531
:1019E000084AC2F898000B6823F01F03034343F032
:1019F0001003C2F89C308B6843F00103C2F8A0309A
:101A0000704700BF00ED00E02DE9F043DFF8608093
:101A100085B00E461F4604464FF00009B14523DA53
:101A20006068D8B13FB1411E08421BD11F2819D9A7
:101A30002368194216D12368019302F085F9A3683F
:101A400003430393D8F89050C5F30725D0B2013D66
:101A5000A84207D801A9FFF7C3FF421C09F10109F9
:101A60000C34DBE76FF01502104605B0BDE8F083DB
:101A700000ED00E0044B0522C3F89420BFF34F8F24
:101A8000BFF36F8F704700BF00ED00E0BFF35F8FC3
:101A9000024B0022C3F89420704700BF00ED00E025
:101AA00010B5034C01232278FFF7AEFF207010BD64
:101AB000D809002008B50B4A00231278FFF7A4FFCD
:101AC00010F1160F07D0084A0021D2F89030C3F366
:101AD0000723984200DB08BDC2F89800C2F8A010A6
:101AE0000130F2E7D809002000ED00E02DE9F043D5
:101AF0005A4B5B4DD3F890302C68C3F307239C42BC
:101B000085B000F2A780FFF7C1FF00200C268442B9
:101B10001AD1544EDFF8449134706846FEF77EFCCB
:101B2000514C524D80460027B84514D133784B496B
:101B30000020D1F89020C2F307229342C0F28480A3
:101B4000FFF798FF002045E0696806FB0011FFF7EA
:101B500047FF0130DBE7009800EB07114FEA071C55
:101B6000CB682340B3F5000F4DD00AD8B3F5001F62
:101B700033D0B3F5800F3BD0B3F5801F13D00137BE
:101B8000D2E7B3F1007F47D0B3F1805F4DD0B3F11E
:101B9000807FF4D150F80C3088684A6802F0D4F89D
:101BA00040F0887009E050F80C3088684A6802F00C
:101BB000CBF840F0885040F43020CDE90123039069
:101BC000D9F890303078C3F30723013B984234D9D9
:101BD0006FF0150005B0BDE8F08350F80C30886850
:101BE0004A6802F0B1F840F0885040F40020E4E781
:101BF00050F80C3088684A6802F0A6F840F000708F
:101C000040F40030D9E750F80C3088684A6802F098
:101C10009BF840F08270D0E750F80C3088684A6832
:101C200002F092F840F48020C7E750F80C30886842
:101C30004A6802F089F82843BFE701A9FFF7D0FE00
:101C40003378013333709AE7C1F89830C1F8A000B7
:101C500001336EE74FF0FF30BCE700BF00ED00E05E
:101C6000444C0008D80900200000F0FF00000211D9
:101C700008B5054801F0F6FB002383F31188BFF394
:101C80006F8F0423184602DFBD51000807B5084ACC
:101C900092E80300CDE9000106488268126822B18B
:101CA0006946904703B05DF804FB6FF05700F9E711
:101CB000D44A0008644700083F280DD800F01F02EE
:101CC00001239340054A1F2894BF5269526B9343E6
:101CD0000CBF012000207047002070470004014025
:101CE00000F01F0201233F2803FA02F307D81F2840
:101CF000044A02D85361002070475363FBE76FF03A
:101D00001500704700040140044B184400230133C0
:101D10008B4200F8012BFADB704700BF3C0000202B
:101D20002DE9F041104F054600264FF001086B7871
:101D3000F4B2A34201D8BDE8F0812B781C442046C0
:101D4000FFF7BAFF68B12046FFF7CAFF57F83430F3
:101D50003BB107EBC40204F01F04516808FA04F019
:101D600098470136E3E700BF0C08002038B50B8820
:101D7000C3F30B030D2B0D46144617D813B96FF0A0
:101D8000850012E0023B0B2B1BD8DFE803F037067F
:101D9000313533311A1A1A1D28284FF4FA402060C1
:101DA0002B68B3F5805F2CD2002038BD03F6B873E2
:101DB000C3F30B03182BE2D8154A22FA03F3DB070F
:101DC000DDD5144B1868EAE700F0E0F80623B0FB15
:101DD000F3F0552358430723B0FBF3F0DFE700F09F
:101DE000D5F80623B0FBF3F0552358434008D6E757
:101DF0000020D4E70848D2E70848D0E74FF4004075
:101E0000CDE7C3F313330133B0FBF3F02060CBE72E
:101E1000110111012C00002000366E01006CDC0263
:101E2000F8B5564F564C00F0CFF8384602F06EF831
:101E300000F058FAA368534AC3F303131578D35C30
:101E400005F01F0503F01F0320FA03F647FA05F516
:101E5000AE4202D2284600F07BFA236823F48023A6
:101E60002360236843F48033236023689803FCD500
:101E7000D4F8943043F00103C4F89430D4F894308B
:101E80009907FBD5FEF748FAD4F8903043F00103E8
:101E9000C4F89030D4F890309A07FBD5FEF75AFA80
:101EA000D4F8983043F00103C4F89830D4F898304F
:101EB0009B07FBD5A36803F00C030C2B18D12368F8
:101EC000580506D4236843F48073236023685905BA
:101ED000FCD5A36823F0030343F00103A360A368C8
:101EE00003F00C03042BFAD1A36823F0F003A360E2
:101EF000236823F08073236023689A01FCD4E3688D
:101F000023F4003343F06053E360E36843F4803329
:101F1000E360E36823F4C003E360E36843F4801301
:101F2000E36000F037F8236843F080732360236890
:101F30009B01FCD5A36823F0F00343F08003A3606A
:101F4000A36843F00303A360A36803F00C030C2B06
:101F5000FAD1A368AE4223F0F003A36002D328466F
:101F600000F0F6F9084B1F60A36823F4E063A36058
:101F7000A36823F46053A3600020F8BD80FE210A0B
:101F800000100240DC5200082C000020004870477E
:101F900000366E010A4AD2F8803023F48073C2F80A
:101FA000803002F5D032074BD1680B4043F4AA438E
:101FB00043F05303D360D36843F08073D36070471A
:101FC000007000400C80FFF9064B9A6D42F0805281
:101FD00082B09A659B6D03F080530193019B02B020
:101FE000704700BF0010024000487047644C000872
:101FF000044BB3F8E0359B020B6000234B6018469E
:10200000704700BF0070FF1F10B5044601690B4800
:1020100083681B68043113B96FF0040010BD984742
:102020000028F9D120690C300122114602F03EFA55
:1020300001F0EAFF00EAE070F0E700BF6447000843
:1020400038B5036905461C6849B101F0DFFF58B196
:1020500028690C3000F000FC6FF0040038BD6369A3
:10206000002B06DB0020F9E7636943F0004363615E
:10207000F8E7034BA36003F18833A360F2E700BFE6
:102080002301674510B50E480368A3B94FF40063F8
:1020900043600C4BB3F8E0404FF6FF739C421DBF0A
:1020A000094BD3F8E045094B4FF4003318BF03EA5E
:1020B0008423DB0A036001230860136010BD00BFA6
:1020C0008C0800200075FF1F0070FF1F00FCFF033D
:1020D0004FF0E0230D4A9969126818699B6900293D
:1020E00008BF1146002B08BF134610F4803F084874
:1020F00001D1994205D20168114401604FF0E021FD
:10210000096900681044C01A704700BFA808002081
:10211000A4080020094B102283F82320084B44F226
:1021200068221A60074B002018604FF0E02344F249
:1021300067225A61072298611A61704700ED00E03A
:10214000A8080020A4080020684620F007018D465A
:1021500019B5FFF7BDFF144B1449D3E900420868D5
:10216000001942F10002C3E90002114A00230B608A
:10217000D2E9004144F26823001BB0FBF3F0434373
:102180001B1941F10001C2E90031EFF31181102365
:1021900083F31288BFF36F8F00F088FFFFF78AFB8D
:1021A000BDE819408546704760000020A408002063
:1021B000580000202DE9F041364E89B1421C0AD169
:1021C0004FF0E022136923F0010313614FF07F43C6
:1021D0003360BDE8F0813568012806DC00240AE0A0
:1021E000431C3568F8D140F2D93040F2DA339842D6
:1021F000A8BF1846441EEFF31187102383F31288FB
:10220000BFF36F8FFFF764FF23494FF0E023D3F84C
:1022100018C0D1E90023801843F10003C1E900038D
:102220001E4B00221A601E4B1A68831A2DD444F2EA
:10223000682E44F2672814FB0E841C44131AB4FB66
:10224000FEF440F226420EFB0433934238BF13469D
:10225000144A934228BF13464FF0E022336094693A
:10226000013B536100239361A445D1E90032ACEBFB
:1022700004000DD20544EB1842F10002C1E900321E
:1022800087F31188BFF36F8FA3E740F22643E3E79C
:10229000C318F1E7A808002060000020A40800206F
:1022A000580000202882FF0038B5EFF31185102375
:1022B00083F31288BFF36F8F084B1C68084B1B68B1
:1022C000E41AFFF705FF85F31188BFF36F8F44F21F
:1022D00068232044B0FBF3F038BD00BF600000204D
:1022E00058000020174B9A6802F00C02042A23D0F1
:1022F0009A6802F00C02082A20D09A6802F00C02B8
:102300000C2A1DD1D968DA68D868DB6801F00301AE
:10231000C3F341630329C2F30312C0F3062003F1A0
:1023200001030CBF084909495B000132B1FBF2F21D
:102330005043B0FBF3F070470448704702487047C1
:10234000002070470010024000366E010024F400A7
:1023500010B52849284A441E8C421368D2F88020C0
:1023600044D803F4C063B3F5007F2FD1D20522D443
:1023700003F1016303F5332398422FD81F4B984292
:102380002ED81F4B98422FD81E4B984294BF002046
:1023900001201D4A136823F00F03034313601368E1
:1023A00003F00F03984223D0136803F00F03181AA9
:1023B00018BF012010BD154B98420FD8144B9842FE
:1023C0000ED8144B98420FD8134BDEE7B3F5806F4D
:1023D00008D1124B984207D8114BD6E70420D8E712
:1023E0000320D6E70020D4E70220D2E70120E1E76E
:1023F0000020DFE77FFE210A0070004080651406A0
:1024000000990D0480CC060200200240000E270730
:10241000804A5D050087930380C3C90100366E01C1
:10242000001BB700F0B5816885B01039054621F072
:10243000070401F088F80B4B6A4603F1100718688F
:102440005968164603C60833BB423246F7D11023FB
:102450006A462146284601F043F8003818BF01209B
:1024600005B0F0BDB64C000830B50D46816887B0A8
:10247000102302AA1039044601F01DF8002802DAE0
:10248000012007B030BD102202A9204601F031FF23
:1024900000283AD11E49102202A802F01DF9002896
:1024A0000CBF012302232B70204601F00EFF0123F5
:1024B00001460DF10702204600F0FDFF0028DFDB9A
:1024C0009DF8073003F00F021B096A702B7101227F
:1024D0000DF10701204601F00CFF10B96B78042BB9
:1024E00003D901236B7000232B71A268183A22F0E4
:1024F0000702083AA91C204601F00EFF0028BFD1B0
:10250000E91C204601F060FFBBE70323CBE700BFD7
:10251000B64C0008F0B5324F460085B00546694616
:1025200057F8260001F056FF044610B1FF2005B011
:10253000F0BD013602A957F8260001F04BFF012833
:1025400008D128482A46492100F09AFF264B0293D9
:102550008DF80C409DF800609DF80870234C002217
:102560002078314601F0B7FE48B36078394601F073
:10257000B2FE20B3A378042B03D09DF80310994238
:102580001DD1E378042B03D09DF80B10994216D18E
:102590002379042B0FD16379023BDBB2022B1AD9CA
:1025A000134B14482A46492100F06AFF6079831EC4
:1025B000022BBCD9BAE79DF802109942EBD0013248
:1025C000032A04F10604CBD10B482A46492100F026
:1025D00057FF0120ABE7094A52F82330E1E700BF7B
:1025E000784C00081D52000803010303EC52000858
:1025F0000B520008675200088B5200086C4C000810
:1026000038B5EFF31185102383F31288BFF36F8F72
:10261000064B9C6801F03CFF85F31188BFF36F8F78
:102620002046BDE83840FFF755B900BFAC08002090
:1026300038B50A4B53F82040013053F82050A542DA
:1026400000D838BD606830B1037EDB0701D401F0EB
:10265000F4FE0834F3E723689847FAE7804C000853
:1026600070B5294B294C2A4D86B0012203201A70DF
:10267000FFF7DEFF0420FFF7DBFF2646AE4204F142
:1026800030040FD300F076FB204CAC4226D300F090
:1026900085FBFDF78DFD1F4A938923F0010393818C
:1026A00006B070BD54F80C3C059354F8103C0493EC
:1026B00054F8143C039354F8183C029354F81C3C0F
:1026C000019354F8203C009354E90A2354E90C0187
:1026D00000F01CF954F8303C5E65CEE7D4E90A23DB
:1026E000B3F1FF3F08BFB2F1FF3F05D052EA03014B
:1026F000206803D100F062F93034C6E7064918308B
:1027000000F0F4FBF8E700BFD9090020984A000860
:10271000984A0008E8000020BD45000870B5002375
:1027200086B00122CDE90423134E144D01930F22EC
:10273000CDE902321249142303FB005506EBC01603
:1027400004464FF4C07000FB04110E4B00954FF48B
:10275000A072304600F0DAF8337C0B4AEE6023F0CA
:10276000040333744FF4046304FB033313442C74E5
:102770006B6006B070BD00BF68000020AC08002090
:102780004012002097440008000A00207FB5002076
:10279000FFF74EFF284B83F30888284C636943F406
:1027A000007363610025F02384F82230E5772576F5
:1027B0006576A57684F82050636A43F4E02363626B
:1027C000FEF78CFFFFF770F84FF0FF33A362E36270
:1027D000FFF78CF9FFF7E8F819481A4C00F0E2F817
:1027E000FDF7E8FD0120FFF723FF0220FFF720FFA0
:1027F00000F0B8FA144B15495C61154B05930123A1
:102800004FF42052CDE90353CDE90155114B00950A
:10281000204600F07BF8237C064623F00403204684
:10282000237401F0A6FE2846FFF778FF094A3146D7
:102830002046FFF71BF800BF4012002000ED00E02B
:1028400068010020E8000020AC080020C013002030
:10285000C25200086126000870B5EFF311861023FC
:1028600083F31288BFF36F8F0468A0421AD0CCB1F3
:10287000D4E9003213605A60237C002523F0020360
:102880002374C4E90055A56004F1180000F0C6FBEC
:102890002046A56701F06DFE31460848BDE870404E
:1028A00001F0A4BED0E902329A4218BF013383601E
:1028B00086F31188BFF36F8F70BD00BFDA09002067
:1028C00013B5EFF31181102484F31288BFF36F8FD7
:1028D000846844B1013C846081F31188BFF36F8F39
:1028E000002002B010BD52EA030406D181F3118822
:1028F000BFF36F8F6FF00F00F3E7CDE900230246BF
:10290000014800F003FAECE7DA0900202DE9F04372
:10291000073285B022F007020E461F4610998181CA
:1029200000F158037F32C0E916330446002322F039
:102930003F020421836001743F2A0F98A073C4E909
:102940000633E37306F14009A2F1400805D883F38A
:102950001188BFF36F8F084602DFB518294620465D
:10296000FEF756FD07300E9B20F00700A066C4E975
:10297000189802930D9B01932D1A0C9B00932A46E5
:102980003B4631462046FEF73FFF00236365044B7C
:102990009B6803B1DB6EE366284605B0BDE8F083B3
:1029A000AC0800200123037483810023C0E918339D
:1029B000C366014B98607047AC08002038B50446E8
:1029C000EFF31185102383F31288BFF36F8F037C1D
:1029D0005B070FD5183000F021FB237C23F00403A4
:1029E0002046237401F0D4FD29460548BDE838404F
:1029F00001F0FCBD85F31188BFF36F8F38BD00BFB8
:102A0000DA090020094A93686FF00A0199670849BA
:102A100058674B6843F080534B60002383F3118861
:102A2000BFF36F8F9368986F704700BFAC080020AA
:102A300000ED00E038B590F91020037C002A014633
:102A400004DA03F07F03037401F05BFD0D4D2A46A9
:102A5000AB6852F8184F944200D004B9EC688B422E
:102A600007D01A7CD20604D1DA897F2A01D9A2695B
:102A70002AB1A34202D0204600F0D6F923466B616A
:102A800038BD00BFAC08002070B590F91020037C61
:102A9000002A2FDBD9062DD11A4C63F07F03224682
:102AA000037452F8183FE169934207D1C0E900214D
:102AB0000860E0610FE09942F8D01B68002BF5D068
:102AC00093F90E6090F90E50AE42F4DD5968C0E9FA
:102AD000003108605860A569954200D005B9E568E5
:102AE000A3681A7CD20606D1DA897F2A03D9AA699B
:102AF0000AB9636170BDAB4202D0284600F094F978
:102B00006561F7E7AC080020034648B9EFF305829A
:102B100032B9064A51699268914201D0FFF772BFFB
:102B200083F31188BFF36F8F704700BFAC0800209C
:102B300038B5184CA168E0690B68814214BF1A4689
:102B4000002249680B605960A368E1692AB9124AFA
:102B5000C3E900210B60E3610AE092F90E5093F99A
:102B60000E00854212DD5168C3E900210B605360FD
:102B7000A569094B9D4200D005B9E568A3689D424F
:102B800002D0284600F050F9656138BD8A42DED097
:102B90001268DBE7AC080020C40800202DE9F047EC
:102BA000002A027C0CBF4FF010094FF0080919EA07
:102BB000020F04460E460F4628D149EA0203D20905
:102BC00046D10374B9F1080F48D04FF00008DFF880
:102BD000F0A0534653F8185F9D4200D00DB9DAF8C3
:102BE0000C50DAF80830AB4202D0284600F01CF94D
:102BF000B9F1100FCAF8145008D0204601F08DF832
:102C0000B8F1000F02D02F48FFF7CCFE2C4B9B6889
:102C1000A3424FD1EFF30583002B4BD1A289D207FA
:102C200011D586F31188BFF36F8F83F31188BFF33B
:102C30006F8F0423184602DFEFF31187102383F30D
:102C40001288BFF36F8F3846BDE8F047FFF7DABE52
:102C500003F07F03037401F054FCB3E7A36813B1DE
:102C6000204601F056FC04F1180000F0D7F9A56DDC
:102C700004F15808A84511D04FF0000A75B1284654
:102C800001F047FC05F1180000F0C8F9C5F878A07C
:102C90002846FFF7F9FEA56DA845EFD1084B9B68C4
:102CA0009C4292D1EFF30588B8F1000818BF4FF0AD
:102CB00001088CE786F31188BFF36F8FBDE8F087BA
:102CC000AC0800206801002070B50F4D2B46064669
:102CD00053F8184F9C4200D004B9EC68AB681A7CDA
:102CE000D20604D1DA897F2A01D9A2692AB1A34286
:102CF00002D0204600F098F823466B613046BDE8CC
:102D00007040FFF701BF00BFAC080020F8B5124BC0
:102D10000C461146114A98681060DDE90676EFF31B
:102D20001182102282F31288BFF36F8F9D682846AC
:102D300001F0F9FBB6F1FF3F08BFB7F1FF3F06D046
:102D400007493A46334605F1180000F0CFF820460F
:102D5000BDE8F840FFF756BEAC080020CC080020C4
:102D6000BD450008024B03F11802C3E90622704773
:102D7000AC080020EFF31181102383F31288BFF316
:102D80006F8F054B9A68D37B013BD37381F3118816
:102D9000BFF36F8F704700BFAC080020EFF31180C6
:102DA000102383F31288BFF36F8F034B9A68D37B92
:102DB0000133D373FFF788BFAC080020014B98683C
:102DC000704700BFAC080020027C12F01F020346CF
:102DD00010D10A4988420DD00949086868B1D989DB
:102DE0007F2909D893F90E20064B1B689A42B8BF79
:102DF0000020704700207047104670476800002090
:102E000030000020D0080020044BC01A044BC01032
:102E10005843044B01221A54704700BFE8010020B8
:102E2000ABAAAAAADA09002070B50C4B0C4C1E7C88
:102E3000FFF7CAFF182303FB06440546204600F0AF
:102E4000EDF8084B00229A553DB12A46EB17204673
:102E50000549BDE8704000F049B870BDAC080020DD
:102E6000E8010020DA090020092E000838B5EFF348
:102E70001185102383F31288BFF36F8F0F4B104A15
:102E80009C681068A04206D1FFF7CEFF85F3118839
:102E9000BFF36F8F38BD00211B7C1160094AD35CE2
:102EA000002BF3D02046FFF78FFF0028EED0237CC5
:102EB000DB0601D1FFF73CFE2046E5E7AC08002029
:102EC000CC080020DA090020024B1868984208BF9D
:102ED0000020704734000020034B1B680BB9FFF73C
:102EE000E3B90020704700BFD4080020B3F1FF3FD2
:102EF00008BFB2F1FF3F2DE9F84F04469946154649
:102F0000984600F081808160EFF31187102383F3EE
:102F10001288BFF36F8FB9F1000FDFF8F4A026DB42
:102F2000FFF7DAFF3B4B1A68B2FA82F245194FEA13
:102F3000521249EBE0795219DAE9005149F10003E4
:102F4000C4E904235519064643EB01084FF0010973
:102F5000FFF7BAFFDFF8C0E0DEF804A00346EBB9E4
:102F6000C4E900EACAF80040CEF8044028E0DAE9F3
:102F700000126FF001035B1A4FF0FF3161EB0202A8
:102F80005B1B62EB0902012B72F10001BCBF012344
:102F90000022C0E904324FF00009D9E7D3E9041C4C
:102FA000D4E904208A4270EB0C0B24DA891A5A689F
:102FB0006CEB0000C3E90410C4E9003214605C60EB
:102FC000FFF782FF84420ED1124B1B685BB9B9F147
:102FD000000F02D1FFF780FF0646304601F009FBE3
:102FE0000021FFF7E7F887F31188BFF36F8F2846BA
:102FF0004146BDE8F88F521A60EB0C005345C4E916
:103000000420ADD01B68AAE70025A846EFE700BF63
:1030100000020020D408002034000020F8B5024649
:10302000EFF31185102383F31288BFF36F8F0168CC
:1030300051B3FFF749FF1C4B5B689A4208D0D1E9B6
:103040000434D2E90476DB1944EB0604C1E9043404
:10305000D2E90031002400264FF0004790420B6077
:103060005960C2E90044C2E9046705D0002085F335
:103070001188BFF36F8FF8BDFFF72EFF01F0B9FA8B
:103080002146FFF797F8F1E7D0E90413B3F1004FB9
:1030900008BF012904D100204FF00041C2E904011A
:1030A0006FF01500E3E700BF340000202DE9F84F72
:1030B000DFF8BC902F4DC9F800000246FFF704FF6F
:1030C0000C4601264FF00047D5E900C14FEAE278EF
:1030D00058B1D0E904AE524578EB0E031CDABAEBD6
:1030E00002036EEB0806C0E9043612EB0C0241EB5A
:1030F0000801C5E9002100252846C9F8005001F063
:1031000078FA2946FFF756F884F31188BFF36F8FDA
:10311000BDE8F84FFFF7AABE1AEB0C0341EBEA71CA
:10312000C5E900314FF0000B4FF01008D0E9011253
:1031300003680B605960C0E900BBC0E9046784F311
:103140001188BFF36F8F9047EFF3118488F31288D3
:10315000BFF36F8FFFF7B8FE18B1D0E90423134314
:10316000E4D0D9F80020A2EB0A02C9F80020ABE7AE
:10317000D40800200002002010B5EFF311841023C2
:1031800083F31288BFF36F8FFFF7A6FE054A03464D
:10319000D2E90001181841EBE37184F31188BFF301
:1031A0006F8F10BD000200202DE9F04F8378D0F81A
:1031B000048015469A0785B0074640F19F80002697
:1031C0000878002800F09C80252808D001F1010A29
:1031D00001363946C047002880F286808AE091F89F
:1031E00001B0BBF1250F01F1020AF1D00024012149
:1031F0001F2C25D8ABF12002102A06D8844B01FAE7
:1032000002F018420ED1032A5AD0ABF13002092A3B
:1032100008D9BBF12A0F33D1630605F1040501D4A7
:1032200044F020041AF801BBBBF1000FE0D139468D
:103230002520C04700285DDB023639465846C9E7DD
:103240007F2CE2D9BBF16C0F29D021D8BBF1680FDC
:103250002CD0BBF16A0F30D0BBF14C0F2DD0ABF1AD
:103260006302122A00F2A580DFE802F02C4EA3A32D
:10327000A3A34EA3A3A3A3A3AD9DA3A331A37700B0
:10328000BBF12E0FDED160063AD444F04004C9E70A
:10329000BBF1740FC6D0BBF17A0FC3D0DFE72206B3
:1032A00048BF44F4007444F08004BBE7E30548BF22
:1032B00044F4007444F48074B4E744F42074B1E737
:1032C0001024AFE715F8040B0136394682E72C6865
:1032D000504B002C08BF1C46A1464B4619F8010B69
:1032E00020B9341B1E190435514669E73946C047D9
:1032F0000028F2DABB7843F00403BB704FF0FF36CE
:10330000304605B0BDE8F08F20061DD5A10545BFAC
:10331000073525F0070555F8040B55F8080B00286C
:103320000DF10409B8BF404249464FF00A02B8BF48
:1033300044F4806401F0E0F96405A0EB090956D477
:103340004C460DF1040B5EE0E20555F8040BE6D5A2
:10335000A3054CBF40B200B2E1E724F01004A4B2D0
:103360000A22200633D5A10545BF073525F00705FC
:1033700055F8040B55F8080B10B924F01004A4B24A
:103380000DF10409494601F0B7F9E306A0EB09097C
:10339000D6D539463020C0470028ABDBBBF1000F43
:1033A0001ED10136CCE744F0100410224FF0780B08
:1033B000D7E74BF02002782A7FF439AFCBF17802BF
:1033C00042F01002CDE708224FF0000BC9E7E305F9
:1033D00055F8040BD0D5A1054CBFC0B280B2CBE7E5
:1033E000023639465846C0470028A9DA82E7013636
:1033F00039462D20F7E7013C39461BF80400C04749
:103400000028FFF677AF002CF5D14E446CE700BFE3
:1034100081280100C7520008704708B500F091F8F4
:10342000002008BD30B5002985B00446154611DBE3
:1034300083688B420ED96368C068194401AA00F002
:1034400097FD28B96268019B9B1A2B60029B6B60F9
:1034500005B030BD6FF02100FAE770477047704744
:10346000002070470FB407B504A951F8040B01916F
:10347000FCF730FF03B05DF804EB04B07047704711
:103480000FB407B504A951F8040B0191FCF722FF12
:1034900003B05DF804EB04B07047002908DB8068D6
:1034A000884205D9401A904234BF0020012070475D
:1034B00000207047704770B516461A4605460C4600
:1034C000FFF7EBFF48B16968E86821448268146837
:1034D0003246A446BDE8704060476FF0150070BDED
:1034E00070B516461A4605460C46FFF7D6FF48B19A
:1034F0006968E8682144826854683246A446BDE899
:10350000704060476FF0150070BD10B50B46044663
:10351000FFF7C3FF40B16168E068194483689B68A6
:103520002BB1BDE8104018476FF0150010BD6FF0CB
:103530005700FBE708B5C0688368DB6898470068F8
:1035400008BDC068704708B5C0688368DB689847E5
:10355000407908BD30B54C680368A34201D2012010
:1035600030BD8A682244934201D30020F8E7D1E9B4
:103570000452954203D36FF00B038B61F5E7CA68E1
:103580001B1B42F835304368086902EBC0025360E8
:103590000B6901330B61E2E737B50C46C0B201A9F4
:1035A0001546FCF741FF00280CDB019850B121467D
:1035B0002A46FCF75FFF04460198FFF77BFF204691
:1035C00003B030BD6FF01504F9E72DE9F0439DB06D
:1035D000DDE926676846249D0C4691469846FDF72E
:1035E00095FE36B1002F04DD3A463146684600F0BC
:1035F000F0FA63892289E76813441F440024A74234
:1036000007D82598694600F00AFB00201DB0BDE8E8
:10361000F0833E1BAE4228BF2E463346424621462B
:103620004846FFF748FF0028F0D132464146684639
:1036300000F0CFFA3444E2E72DE9F7430E4617468F
:103640009946044628B94FF0FF38404603B0BDE81C
:10365000F0830029F7D0002AF5D0CB680D891D44EE
:1036600004230DEB030229463846FFF724FF80466A
:103670000028E8D1BDF80410738946F6081291427B
:1036800025D1BDF806109942DDD104230DEB0302CC
:1036900029443846FFF70FFF0028D4D1BDF8042095
:1036A00046F607139A42CED1C4E900679DF8283048
:1036B000A4F80890A3727389BDF806202B44E36038
:1036C000738913442B44043563612561BDE7002BE6
:1036D000E4D0B8E72DE9F3410E4617461D460446EF
:1036E00020B94FF0FF3002B0BDE8F0810368002B35
:1036F000F7D04368002BF4D04FF6FF78D4E90413D9
:10370000994215D223685B8923B1E3688B4204BFD9
:1037100004312161042360680DEB0302FFF7CBFE47
:103720000028DED1A37A2BB1D4E903329A4201D327
:103730000120D8E72389BDF80610434501F10402B2
:1037400003D0BDF804C09C450BD115B1BDF80430C1
:103750002B80236904333360398023691344236148
:10376000C1E7236913442361C8E748B103683BB14B
:1037700043682BB1C068884294BF00200120704785
:103780004FF0FF30704700F0A7BF10B50446FFF7B9
:10379000D1FE00F086F8A368984201D900F0E4FA5F
:1037A000181A10BD70B50D46044600F08EFD2A466D
:1037B000A0F1080104232046BDE87040FFF77BBE5E
:1037C00013B50446019100F080FD0423A0F1080127
:1037D0000DEB0302204600F0BBFD02B010BD00F06F
:1037E000E2B901292DE9F341174601D900F0BCFAED
:1037F0002C2303FB0104D4F82080B8F1000FF5D08E
:10380000E36826891E4404230DEB0302314640463B
:10381000FFF751FE054620B10125284602B0BDE85C
:10382000F081BDF80420648946F608139A421AD143
:10383000BDF806309C4201D00325EEE704230DEBD2
:103840000302A1194046FFF736FE0028E4D1BDF877
:10385000042046F607139A42EED1BDF80610214423
:1038600031443960D9E7002CF1D0E5E713B51822CF
:1038700001290346019208460AD15A6A03F1280435
:1038800001A9FFF789FE08B9019B236002B010BDB2
:10389000022903D11A6D03F15404F1E70120F5E781
:1038A0007047482358433030704773B50C4605467F
:1038B0001646FFF73FFEA04203D92846FFF73AFE1F
:1038C0000446A9684823303903FB14116A46284688
:1038D000FFF7A8FD0028A4BF009B336002B070BDB5
:1038E0002DE9F7431F4683688B4206460D469146F5
:1038F00033D95B1A934230D307B36A46FFF792FD80
:10390000041E2CDB013DDDF800804D446A4629464B
:103910003046FFF787FD041E21DBDDE900953046C8
:103920002A464946FFF7F1FD041E18DBFFF797FD15
:1039300077B1C84513D209F1FF35E7E701396A4687
:103940004944FFF76FFD041E09DBDDF80080DDE769
:103950004D44A84503D30135D8E74FF0FF34204646
:1039600003B0BDE8F08310B412B110BCFFF7B8BFCC
:10397000104610BC7047002382681946FFF7F3BF5A
:1039800008B52C2303FB0101086A08B900F0ECF923
:10399000BDE80840042200F0ACBCF8B513460F4661
:1039A0001646002102460546FDF702F9044650B9C5
:1039B000334605F12C0201212846FDF7F9F810B134
:1039C000002F18BF04462046F8BD00207047002194
:1039D00010B504460846FCF75DFC04F12001C0B2B6
:1039E000FCF722FD40B90121FCF754FC04F14C0125
:1039F000C0B2FCF719FD08B100F0B6F910BD10B562
:103A00000446C06C08B1FFF755FD206A18B1BDE847
:103A10001040FFF74FBD10BD6022002100F054BEE2
:103A20004379012B07D10368012B04D10079431E90
:103A300058425841704700207047F7B5056A07465D
:103A400028460E46FFF7A1FEF96D0446304600F009
:103A500096F804442846FFF76DFD07462846FFF711
:103A600072FD072201460DF1010000F02DFE3379B1
:103A70008DF800306A463B4621462846FFF730FD68
:103A8000003818BF012003B0F0BD13B50C4601AAE1
:103A9000C16D2046FFF709FF002809DB0199A268E4
:103AA0000123521A2046FFF75EFFC00F02B010BD7F
:103AB0000120FBE737B50C46C06C69461546FEF79A
:103AC000D3FC024608B100F04FF9E979012904D08E
:103AD000204600F093FC0028F5D19DF80330012B1F
:103AE00004D1204600F069FC0028ECD1A9682046EA
:103AF000FFF766FE0028E6D12046FEF793FC00287B
:103B0000E1D103B030BD73B50C460646FDF74AF966
:103B1000E06028B3022801D1356A0DB900F024F91C
:103B2000224631462846FDF79BF8D0B9284600F0DA
:103B3000CCFB012301460DF107022846FFF7BBFC31
:103B400088B901220DF10701284600F0D2FB10B11F
:103B500001238DF807309DF8073003F00F03E37160
:103B6000002002B070BD0120FBE7436A00205A68C4
:103B7000034613448B4200F10100FAD3704710B59D
:103B800043790279012B1ABF18234B43002302F11A
:103B9000FF3201FB0233026814BF4C000C46013AAD
:103BA00004FB023010BD10B50446C06DFFF779FE6E
:103BB000636A5B685A1E024459421140A26A013A84
:103BC0005A43501A626D53435B1A984228BF1846F5
:103BD00010BDF8B50C4610B1F9B10AB90120F8BD15
:103BE0008D1800F128060027AC42F7D0836E5A1CCE
:103BF0008266034414F8011B83F828103F2AF3D986
:103C00003146FDF799FAD0E9083213F5007342F115
:103C10000002C0E908328766E6E70846DFE7F8B544
:103C20000C46054600284CD000294BD08B6ED1E9BC
:103C30000821D800121841F10001581C2344C4E99E
:103C4000082138284FF08002A0664FF0000783F863
:103C5000282004F128060BD9C0F14002394630442F
:103C600000F032F820463146FDF766FAA76638467E
:103C7000C0F138020021304400F026F8236A626A5D
:103C80001BBA12BAC4E9182331462046FDF754FA8C
:103C90002B1D211F243551F8042F03F8012C100E81
:103CA00003F8040C100C03F8030C100A03F8020CC0
:103CB0000433AB42EFD120467022002100F004F81B
:103CC0000120F8BD0846FCE700F0FEBC10B5036A11
:103CD0000446D8688368DB689847E36CD8688368D3
:103CE000DB689847012010BD00F0EEBC00F0DEBCA0
:103CF000012801D1EFF30583FEF782BC014600687D
:103D0000FFF7F6BF08B5FDF77FFBBDE80840FDF7FC
:103D1000D1BD00210120FFF7EBBF6FF08500704798
:103D200061B662B680F31188BFF36F8F704772B6C9
:103D3000002383F31188BFF36F8FBFF34F8F30BF22
:103D400062B6BFF36F8F7047202809D9B0F1004FDA
:103D500008D80138B0FA80F0C0F11F004000704769
:103D6000082070473E20704708B5FDF781FF08B571
:103D7000062201210020FDF7C7FF00221146062080
:103D8000FDF700FD012108460722FDF7BDFF0022D7
:103D900011460720FDF7F6FC082201210220FDF75D
:103DA000B3FF002211460820FDF7ECFC0922012197
:103DB0000320FDF7A9FF002211460920FDF7E2FCD0
:103DC0000A2201210420FDF79FFF002211460A204C
:103DD000FDF7D8FC052108461722FDF795FF0022C4
:103DE00011461720FDF7CEFC282206210A20FDF7F8
:103DF0008BFF002211462820FDF7C4FC002008BDDF
:103E00000B88C3F30B0303F6B872C2F30B02182A34
:103E100082B014D803F1804303F5043348681A686C
:103E200002431A600B88C3F30B0303F1804303F5CD
:103E3000043300201B680193019B02B070476FF0B0
:103E40008500FAE70B88C3F30B0303F6B872C2F3DD
:103E50000B02182A9FBF03F1804303F5043349681E
:103E60001A689DBF8A4300201A606FF08500704772
:103E70000D2809D843F66E73C34013F0010F0CBF31
:103E80006FF08500002070476FF08500704770B5B7
:103E900008884A68C0F30B0094B2C2F30445FFF7E8
:103EA000E7FFA0B9FF2A11D004F18041C2F34156C7
:103EB00001F5043101360123B3400C68013BAB40EE
:103EC000120E24EA0303AA4013430B6070BD6FF087
:103ED0008500FBE70888C0F30B0008B500F6B8734F
:103EE000C3F30B03182B0AD800F1804000F504300F
:103EF0004B68026893430CBF0220012008BDFFF706
:103F0000B7FF00280CBF02200120F7E77047F7B584
:103F10001C461646002382682360A36053690D4641
:103F200001AA69469847019B5A1E01921BB96FF07E
:103F3000150003B0F0BD0098A2684768216867606B
:103F400085B9B31AD0F800C0634528BF63461A4448
:103F500003FB07112160A26002689A4206D808306C
:103F60000090E0E76B1AB3FBF7F3EBE70020E0E724
:103F700013460022FFF7CBBF2DE9F047836886B0D8
:103F80005B698846914601A902AA98470024A24687
:103F90002546029BAB4202D806B0BDE8F087019FE0
:103FA00007EBC50700267B6804933A68B2420AEB28
:103FB000060302D801359A46EBE703940593494678
:103FC00003A8C0470028E7D0049B01361C44ECE757
:103FD0004FF0FF324FF0FF330C30FEF771BC70B57D
:103FE0001C461546002322460E4600F0AAF840B1B2
:103FF0002CB1224606F10061284600F057FB002054
:1040000070BD6FF01500FBE70020704773B50646E2
:104010004FF4FA720023684600F002FB33691B6814
:104020001A6944F2FA310A40DDE9004513D01A69F1
:104030000A401A616FF0040002B070BD002AF9D185
:1040400022462B46684600F010FBDDE900321343A0
:104050000CBF0122002233691B68186910F48030FC
:10406000ECD1E9E770B5012305460E46144600F091
:1040700068F8002834D074B32869FFF7A9FF00213D
:104080002846FDF7DDFF40BB31462246284600F0BA
:1040900074F806462B691B681A6852050FD51A6812
:1040A00022F480621A601A6842F480521A601A6818
:1040B00022F480521A601A6842F480621A60012168
:1040C0002846FDF7BDFF002E14BF3446044628697C
:1040D0000C30FEF7C1FB204670BD6FF00406D9E737
:1040E0006FF01504F7E7F8B51C4617460123224682
:1040F00005460E4600F025F800B3D4B12869FFF755
:1041000067FF00212846FDF79BFFA0B931462346F3
:104110003A46284600F08BF8064601212846FDF76E
:104120008FFF002E14BF3446044628690C30FEF77A
:1041300093FB2046F8BD6FF00406EEE76FF0150420
:10414000F7E77FB506460D4614461BB141EA020368
:104150005B0710D101AA29463046FFF709FF50B985
:10416000013C01AA61193046FFF702FFB0FA80F066
:10417000400904B070BD0020FBE7013AF8B50746DE
:104180000D4600205618AE4200D2F8BD3B691C68AF
:104190006369002B48DB3846FFF738FF0028F4DB63
:1041A000636943F002036361636923F4FC73636131
:1041B0006369EA0A43EAC2036361636943F48033D3
:1041C000636138466369FFF721FF23685A050FD5FD
:1041D000236823F480632360236843F480532360BF
:1041E000236823F480532360236843F480632360AF
:1041F00023689B050FD5236823F40073236023688D
:1042000043F400632360236823F40063236023687E
:1042100043F4007323606369002823F002036361A1
:10422000B3DB05F50065AEE76FF00400ADE72DE9FF
:10423000F84F0546002016469846044601F10067EF
:10424000A04510D924F007033344E210D3F804A0AA
:104250002B6956F832B0D3F80090D9F81430002BFF
:1042600003DA6FF00400BDE8F88F2846FFF7CEFEB2
:104270000028F8DB3A59013207EB040302D15A68EF
:10428000013202D05BEA0A02EBD1D9F8142042F0E5
:104290000102C9F81420D9F81420C3F800B0284648
:1042A000C3F804A0FFF7B2FED9F81430002823F0B9
:1042B0000103C9F81430D6DB0834C1E74FF0E0221F
:1042C000136923F00103136170478068183820F0E8
:1042D000070010387047042809D0052803D1481E6C
:1042E00018BF01207047431A5842584170470120B7
:1042F000704738B515460C4661B15AB1FFF723F93E
:104300002544214611F8013B834203D1A942F9D14A
:10431000012038BD0020FCE738B50C4601231146CA
:1043200022460546FFF7C7F800280FDB0122214689
:104330002846FFF7DEFF18B103232370002038BDA5
:104340002378012B14BF02230123F6E70120F6E7AF
:104350002DE9F3471D4606460F469046FFF7EAF85B
:104360006C1E044440420440082C01D9FFF7FCFCB9
:104370003046FFF7E8F82A4682464146684600F094
:1043800095F9621B51460DEB050000F09DF923469F
:104390006A4639463046FFF7A3F8003818BF0120B7
:1043A00002B0BDE8F08707B501238DF8042001AA0B
:1043B000FFF7CEFF03B05DF804FB816818390122D6
:1043C00021F00701FFF7EFBF8268183A22F00702D9
:1043D000FFF7A2BF13B50C46C0B201A9FCF724F841
:1043E00050B921460198FEF73FF804460198FFF7BF
:1043F00061F8204602B010BD0124FAE70E2A13B579
:10440000044601D9FFF7B0FC0E29FBD841EA02119E
:104410008DF80710FFF759FF012301460DF1070240
:104420002046FFF795FF02B010BD8168183921F0D2
:10443000070101220839FFF7B6BF10B543690446EA
:104440003BB90020E268537843F0010353704042C7
:1044500010BD98470028F4D00028B8BF4042E36858
:10446000FF28A8BFFF201870ECE740B1C368587858
:1044700010F001001EBF1878B0FA80F040097047B4
:10448000EFF31183102383F31288BFF36F8FFEE7DE
:1044900008B5FFF7F5FF08B51024EFF3118384F397
:1044A0001288BFF36F8FFFF742FCF6E73AB18A42FA
:1044B00005D3C0E90212C0E90000002070476FF088
:1044C0001500704738B58589EFF31181102282F30A
:1044D0001288BFF36F8F037C13F0080404D081F3BC
:1044E0001188BFF36F8F38BD0122FEF757FBEB0732
:1044F000F9D584F31188BFF36F8F0423184602DFC8
:10450000F1E7D0E9003213605A600023C0E90033BC
:10451000704708B5FFF7F5FF037C23F0020303742F
:104520000023836008BD38B504460D46FEF782FAC5
:10453000237C43F002032374D5B1A5602B689D4210
:1045400009D16B68C4E900531C606C6010E06A68B4
:104550009A42F6D01B68002BF3D093F90E1094F911
:104560000E209142F3DD5A68C4E9003214605C60A9
:1045700038BD10B5EFF31184102383F31288BFF315
:104580006F8FFEF781FA84F31188BFF36F8F10BD30
:10459000FEF77ABA08B5037C13F0280F01460CD158
:1045A00083680BB1FFF7B5FF0B7C23F004030B749A
:1045B0000846BDE80840FEF767BA08BD10B5EFF33E
:1045C0001184102383F31288BFF36F8FD0E9042383
:1045D000B3F1004F08BF012A04D084F31188BFF360
:1045E0006F8F10BD1838FFF7D5FFF6E70846FEF7C6
:1045F0008BBA08B50246FEF767FC70B1D0E904310A
:104600009B1A61EBE272B3F1004F72F1000104DA20
:10461000002AACBF1846002008BD6FF00040FBE741
:10462000B3F1FF3F08BFB2F1FF3F70B506461D462C
:10463000144614D01A4316D0002B08DBFEF79CFD5D
:10464000041941EB0501C6E90041304670BD6FF029
:1046500001031C1B4FF0FF3363EB0501F3E74FF041
:10466000FF342146EFE70024FBE7B3F1FF3F08BF2B
:10467000B2F1FF3FF8B5074616461C4610D054EA83
:10468000020311D0FEF778FDB0420A46A14103466D
:104690000AD2F31A64EB0204C7E900343846F8BDC5
:1046A0004FF0FF331C46F7E70023FBE70A44914233
:1046B00000F1FF3300D1704710B511F8014B03F83A
:1046C000014F9142F9D110BD02440346934200D1FB
:1046D000704703F8011BF9E710B501390244904215
:1046E00001D1002005E0037811F8014FA34201D069
:1046F000181B10BD0130F2E7F0B5C2F137050446D2
:10470000EDB202F01F020846B4FBF2F602FB1641BE
:10471000CBB2092988BF5B19274688BFDBB230338B
:0C472000BA4200F8013B3446EED9F0BD6F
:10472C0000000000644700080503000800000000BA
:10473C0000000000804700086F3D000800000000EA
:10474C001521000800000000000000009C47000834
:08475C00B90200080000000092
:10476400E451000800000000B04A00084E00002098
:1047740000000000211E000800000000C6510008CF
:1047840000000000000000004C00002000000000B9
:104794008D1C000800000000F1510008000000001A
:1047A400984A00085000002010000020092000084A
:0447B4000000000001
:1047B80000000000133D000800000000133D000841
:1047C80000000000133D000800000000133D000831
:1047D80000000000133D000800000000133D000821
:1047E800DA520008211D0008D8520008211D0008CF
:1047F800D6520008211D0008D4520008211D0008C7
:10480800D2520008211D000800000000133D0008D6
:1048180000000000133D000800000000133D0008E0
:1048280000000000133D000800000000133D0008D0
:1048380000000000133D000800000000133D0008C0
:1048480000000000133D000800000000133D0008B0
:1048580000000000133D000800000000133D0008A0
:1048680000000000133D0008D0520008211D000878
:1048780000000000133D000800000000133D000880
:1048880000000000133D000800000000133D000870
:1048980000000000133D000800000000133D000860
:1048A80000000000133D000800000000133D000850
:1048B80000000000133D000800000000133D000840
:1048C80000000000133D000800000000133D000830
:1048D80000000000133D000800000000133D000820
:1048E80000000000133D000800000000133D000810
:1048F800CE520008211D000800000000133D0008EA
:1049080000000000133D000800000000133D0008EF
:1049180000000000133D000800000000133D0008DF
:1049280000000000133D000800000000133D0008CF
:1049380000000000133D000800000000133D0008BF
:1049480000000000133D000800000000133D0008AF
:1049580000000000133D000800000000133D00089F
:1049680000000000133D000800000000133D00088F
:1049780000000000133D000800000000133D00087F
:1049880000000000133D000800000000133D00086F
:1049980000000000133D000800000000133D00085F
:1049A80000000000133D000800000000133D00084F
:1049B80000000000133D000800000000133D00083F
:1049C80000000000133D000800000000133D00082F
:1049D80000000000133D000800000000133D00081F
:1049E80000000000133D000800000000133D00080F
:1049F80000000000133D000800000000133D0008FF
:104A080000000000133D000800000000133D0008EE
:104A180000000000133D000800000000133D0008DE
:104A280000000000133D000800000000133D0008CE
:104A380000000000133D000800000000133D0008BE
:104A480000000000133D000800000000133D0008AE
:104A580000000000133D000800000000133D00089E
:104A680000000000133D000800000000133D00088E
:104A780000000000133D000800000000133D00087E
:104A880000000000133D000800000000133D00086E
:104A9800DF3F0008E740000865400008E91F0008FC
:104AA800F11F000885200008013E0008453E000867
:104AB800000000006D1D0008D53E00080000000041
:044AC8008F3E000815
:084ACC008F4D000803000000FB
:104AD400600000000100000001000000020000006E
:104AE4000400000000000000000000000088000036
:104AF4009C470008010000000088000000C000007E
:104B04009C470008020000000048010000A80000C3
:104B14009C4700080300000000F0010000100000A2
:104B24009C47000801000000020000000100000092
:104B340002000000982F8A4291443771CFFBC0B520
:104B4400A5DBB5E95BC25639F111F159A4823F9254
:104B5400D55E1CAB98AA07D8015B8312BE853124AD
:104B6400C37D0C55745DBE72FEB1DE80A706DC9B6E
:104B740074F19BC1C1699BE48647BEEFC69DC10F1A
:104B8400CCA10C246F2CE92DAA84744ADCA9B05C56
:104B9400DA88F97652513E986DC631A8C82703B019
:104BA400C77F59BFF30BE0C64791A7D55163CA0627
:104BB40067292914850AB72738211B2EFC6D2C4D33
:104BC400130D385354730A65BB0A6A762EC9C28121
:104BD400852C7292A1E8BFA24B661AA8708B4BC2B7
:104BE400A3516CC719E892D1240699D685350EF4E1
:104BF40070A06A1016C1A419086C371E4C77482798
:104C0400B5BCB034B30C1C394AAAD84E4FCA9C5B0D
:104C1400F36F2E68EE828F746F63A5781478C8845E
:104C24000802C78CFAFFBE90EB6C50A4F7A3F9BE40
:104C3400F27871C6000000200000000000000B069E
:104C4400020000004C4C000800000008AE510008AF
:104C54002000020200000020B65100081C000B11C5
:104C64000800000000FF0000B1520008B65200081E
:104C7400BB52000801000000020000002C4700089D
:104C84002C4700084C470008544700085C470008BC
:104C94006447000801000200100011001200200007
:104CA40021002200230024003000310032003300B0
:104CB400FFFF77C295F360D2EF7F3552500F2CB6C9
:104CC400798025633A205374617274696E67206237
:104CD4006F6F746C6F616465720A0025633A2055C6
:104CE4006E61626C6520746F2066696E6420626F09
:104CF4006F7461626C6520696D6167650A00256384
:104D04003A20426F6F746C6F6164657220636861EE
:104D1400696E6C6F61642061646472657373206F83
:104D240066667365743A20307825780A0025633AFC
:104D340020496D6167652076657273696F6E3A20EC
:104D44007625642E25642E25640A0025633A204ABC
:104D5400756D70696E6720746F207468652066696C
:104D640072737420696D61676520736C6F740A00D7
:104D740025633A204E657665722073686F756C649E
:104D84002067657420686572650A006D6375626FDB
:104D94006F740025633A20696E76616C69642066DD
:104DA4006C6173682049442025640A002A2A2A2059
:104DB4005573696E67205A6570687972204F532065
:104DC4006275696C642076342E342E302D32373778
:104DD400332D6734343234616136383165306220C2
:104DE4002A2A2A0A0025633A204661696C656420F0
:104DF400746F2072656164207374617475732066C6
:104E0400726F6D2025642C206572722025640A0A55
:104E1400007072696D617279007365636F6E6461AD
:104E240072790025633A20436C6561726564206978
:104E34006D616765202564207072696D61727920E7
:104E4400736C6F7420747261696C6572206475652B
:104E540020746F20737475636B2072657665727449
:104E64000A0025633A20496D61676520696E2074E4
:104E7400686520257320736C6F74206973206E6FCE
:104E8400742076616C6964210A0025633A202564E4
:104E94002073746174757320777269746520666118
:104EA400696C7320706572666F726D696E672074C9
:104EB400686520737761700A0025633A204661694A
:104EC4006C656420746F206F70656E20666C61730E
:104ED400682061726561732C2063616E6E6F74204B
:104EE400636F6E74696E75650A0025633A204661C6
:104EF400696C65642072656164696E6720736563BB
:104F0400746F72733B20424F4F545F4D41585F4959
:104F14004D475F534543544F52533D2564202D2044
:104F2400746F6F20736D616C6C3F0A0025633A20C7
:104F34004661696C65642072656164696E672069A5
:104F44006D61676520686561646572733B20496DB6
:104F54006167653D25750A0025633A204661696CE1
:104F640065642072656164696E6720626F6F742086
:104F74007374617475733B20496D6167653D257574
:104F84000A0025633A2070616E6963210A00256373
:104F94003A20446574656374656420696E636F6E5A
:104FA40073697374656E7420737461747573210A04
:104FB4000025633A2043616E6E6F742075706772CA
:104FC4006164653A206E6F74206120636F6D706157
:104FD4007469626C6520616D6F756E74206F6620F4
:104FE400736563746F72730A0025633A2043616EBC
:104FF4006E6F7420757067726164653A206D6F72AC
:105004006520736563746F7273207468616E2061C8
:105014006C6C6F7765640A0025633A2043616E6E99
:105024006F7420757067726164653A206E6F7420C6
:1050340073616D6520736563746F72206C61796F41
:1050440075740A0025633A2043616E6E6F7420758F
:105054007067726164653A20736C6F74207772694B
:1050640074652073697A657320617265206E6F744C
:1050740020636F6D70617469626C650A00626164BB
:1050840000676F6F6400756E736574005072696DAC
:1050940061727920696D6167650025633A20257323
:1050A4003A206D616769633D25732C2073776170C5
:1050B4005F747970653D307825782C20636F707942
:1050C4005F646F6E653D307825782C20696D61676B
:1050D400655F6F6B3D307825780A005365636F6EAA
:1050E4006461727920696D6167650025633A2042C5
:1050F4006F6F7420736F757263653A207072696D97
:1051040061727920736C6F740A0025633A20426FD0
:105114006F7420736F757263653A206E6F6E650AE3
:105124000025633A205374617274696E6720737743
:105134006170207573696E67206D6F766520616C90
:10514400676F726974686D2E0A0025633A204E6F8A
:105154007420656E6F75676820667265652073706C
:1051640061636520746F2072756E2073776170209F
:10517400757067726164650A0025633A207265710F
:10518400756972656420257520627974657320627F
:105194007574206F6E6C79202575206172652061AD
:1051A4007661696C61626C650A00464C4153485FE4
:1051B40030005352414D5F300061626F7274282990
:1051C4000A00696E746572727570742D636F6E7403
:1051D400726F6C6C65724034303031303430300072
:1051E40072636340343030323130303000666C6189
:1051F40073682D636F6E74726F6C6C6572403430BB
:10520400303232303030004255473B2063616E27E4
:10521400742068617070656E0025633A205365637D
:105224006F6E6461727920696D616765206F6620B5
:10523400696D616765207061697220282564292081
:10524400697320756E726561636861626C652E2096
:10525400547265617420697420617320656D707483
:10526400790A0025633A20496D61676520696E6497
:1052740065783A2025642C20537761702074797006
:10528400653A2025730A0025633A20496D616765F4
:1052940020696E6465783A2025642C205377617008
:1052A40020747970653A206E6F6E650A00746573B8
:1052B40074007065726D00726576657274006D615C
:1052C400696E00286E756C6C29000A0605050401D8
:1052D40003010201010100010000000000000000C0
:1052E400010203040607080904010403040204017B
:0C52F40004010403010403040104000091
:1053000061340008E84A000801000000FFFFFFFFC9
:1053100000200240480000000001000000000000E2
:105320000000000000000000000000000024F40065
:10533000C80000003400002034000020FFFFFFFF01
:0C534000FFFFFFFFFFFFFFFFFFFFFFFF6D
:08534C00000000000000000059
:0453540015E015E06B
:0400000508001709CF
:00000001FF
